:1000000012C02BC02AC029C028C027C01CC125C0CF
:1000100024C0D9C022C021C020C01FC01EC01DC026
:100020001CC01BC01AC011241FBECFE5D4E0DEBF28
:10003000CDBF10E0A0E6B0E0EAE8F0E102C0059034
:100040000D92A039B107D9F710E0A0E9B0E001C0E6
:100050001D92A43AB107E1F7FDC1D2CF86E886B977
:1000600017B887B1806C87B9369A349BFECF20E0F1
:1000700030E040E0369A349BFECF84B195B1280F32
:10008000391F4F5F4430B0F33798C9019695879573
:1000900096958795089568E28ED7E0E6F0E0E90F3F
:1000A000F11D8081809599270895C39A0895C3987A
:1000B0000895809192008823D1F480919400882340
:1000C00031F080919D006AE076D7892F01C081E1EF
:1000D000E2DF8093990080919400882329F0809139
:1000E0009D006AE068D701C081E1D5DF58C08091EA
:1000F0009200813009F055C080919100813019F54E
:1001000080919600992701966AE070E060D79C0183
:1001100080919400882319F4C901449601C0C90153
:10012000BADF8093990080919600893048F08091E1
:100130009600992701966AE070E049D7CB0101C08B
:1001400081E1A9DF2CC0809191008230A9F48091D7
:1001500096006AE030D7892F8C5E9DDF80939900EE
:10016000809196008A3028F0809196006AE023D72B
:1001700001C081E190DF13C0809196006AE01BD737
:10018000892F89DF80939900809196008A3028F02A
:10019000809196006AE00FD701C081E17CDF8093F7
:1001A0009A0080919100823069F48091A0008823A8
:1001B00041F080919400813011F477DF089577DF6A
:1001C000089575DF08951F920F920FB60F921124B4
:1001D0002F933F934F938F939F93EF93FF938BEFC7
:1001E00082BF80919000992701969C012E7F3370E9
:1001F000821B930B8093900045B3437080919000D5
:10020000282F33272C5F3F4F81E090E002C0880FFA
:10021000991F2A95E2F780958073482B45BB809102
:100220009000E82FFF27E756FF4F808182BBFF91A8
:10023000EF919F918F914F913F912F910F900FBE12
:100240000F901F9018951F920F920FB60F921124C6
:100250002F933F934F935F936F937F938F939F93CE
:10026000AF93BF93EF93FF9380919300882309F09E
:100270004EC080919100823029F58091A0008823A2
:1002800031F08091A00081508093A0001BC080912C
:100290009C00882321F080919C00815011C08091A6
:1002A0009F00882379F080919F00815080939F0068
:1002B00080919F00882331F08FE08093A0008EE131
:1002C00080939C0080919100813009F58091950088
:1002D000882321F08091950081500AC0809196007A
:1002E000882349F0809196008150809396008BE39B
:1002F000809395000CC082E0809391008FE0809302
:10030000A0008EE180939C0083E080939F0083B3E4
:1003100099278E70907020919B0033278217930746
:1003200051F4809198008A3F80F4809198008F5F0B
:10033000809398000AC080919B008093970083B3BC
:100340008E7080939B00109298008091980083306B
:1003500049F58091970090919B0089278093A30095
:100360002091A30080919B00992780959095282348
:1003700021FF1EC080919200882371F481E0809358
:100380009200809391008BE38093950080919D0073
:100390008150809396000CC01092920010929100B0
:1003A00086DE06C080919800843010F0809198001D
:1003B000809193006AE0FFD5992339F480919200EF
:1003C000882319F481E080939E0090E0809193004F
:1003D000893108F091E090939400809193009927DF
:1003E000019662E370E0F3D58093930062DEFF91A3
:1003F000EF91BF91AF919F918F917F916F915F919D
:100400004F913F912F910F900FBE0F901F90189515
:100410009FEF91BB92BB8CE384BB8EE085BB97BB07
:1004200018BA85E083BF8BEF82BF1FBC8DE08EBD05
:1004300080E590E09BBD8ABD1DBC1CBC81E189BFED
:100440001092900083B38E7080939B00109298005E
:1004500078940895CFE5D4E0DEBFCDBFD9DF809199
:100460009E008130E1F7FADD8C01C801AA2797FDD3
:10047000A095BA2FBC01CD011BD317FF05C020E00A
:1004800030E040E857E473D120E030E040E752E448
:10049000C8D1DC01CB0120E030E040E85AE3BC01E8
:1004A000CD01BFD1DC01CB0120E030E040E85FE3CB
:1004B000BC01CD015CD1DC01CB01BC01CD010FD071
:1004C000DC01CB018093A10080919200882321F46C
:1004D0008091A10080939D0010929E00C0CFEF926A
:1004E000FF920F931F937B018C0120E030E040E0EE
:1004F0005FE4ADD288238CF020E030E040E05FEC98
:10050000C801B70134D1DC01CB01BC01CD0131D32D
:10051000605070408040904803C0C801B70129D3A3
:100520001F910F91FF90EF900895A0E0B0E0EAE9ED
:10053000F2E074C58C017B015A01DC018C918230A0
:1005400058F0FB019081923010F4A7010BC1843068
:1005500029F4943009F4A6C0A80104C19430A9F389
:10056000923009F4A9C0823081F3F801C280D380AF
:10057000FB0162817381F8012481358146815781B5
:10058000F7016480758086809780C601861B970B73
:1005900097FDD8C080970CF46CC06C157D050CF0ED
:1005A000ADC0662477244301F8016181F7018181A0
:1005B000681709F499C0662309F491C0621A730A96
:1005C000840A950AA401930157FDC0C0F501118268
:1005D000B60119012A0179018A0139014A010894F9
:1005E0006108710881089108FFEF6F16FFEF7F0621
:1005F000FFEF8F06FFE39F06F0F4A8019701220F9B
:10060000331F441F551F19012A01B6016150704064
:100610006B0179018A0139014A0108946108710866
:10062000810891088FEF68168FEF78068FEF8806A4
:100630008FE3980610F383E0D5018C9357FC64C0D8
:10064000F501248335834683578373836283A50131
:1006500089C06F5F7F4FD401C30181709070A0701B
:10066000B0709694879477946794682A792A8A2A36
:100670009B2A6C157D056CF311C00894C11CD11C1C
:10068000DA01C90181709070A070B07056954795DD
:1006900037952795282B392B4A2B5B2BC616D70667
:1006A00064F382CFF8019181FB018181981709F4ED
:1006B00053CF48E850E056C0823009F04DCF88E073
:1006C000DA01F80101900D928A95E1F7F801818134
:1006D000FB0191818923FA018183A50143C0261979
:1006E00037094809590970CFF5016183B601260D14
:1006F000371D481D591D19012A019DCF6B0120E0AE
:1007000030E040E050E050CFD201C101B695A7954E
:100710009795879521E030E040E050E02222332297
:1007200044225522282A392A4A2A5B2AF5012482A2
:100730003582468257820894C11CD11CD382C28262
:10074000A50110C0909581959F4F24CF81E0F501C0
:100750008183B60150954095309521953F4F4F4F7D
:100760005F4F37CFCA01E2E1CDB7DEB773C4A0E275
:10077000B0E0ECEBF3E060C4DC01CB01898F9A8F31
:10078000AB8FBC8F2D8F3E8F4F8F58A3BE016F5FF5
:100790007F4FCE01499622D38E01075F1F4FB801CC
:1007A000CE014D961BD3AE014F5E5F4FB801CE0117
:1007B0000196BBDE2DD2DC01CB01BC01CD01E4E012
:1007C000A09656C4A0E2B0E0E7EEF3E035C4DC0149
:1007D000CB01898F9A8FAB8FBC8F2D8F3E8F4F8F20
:1007E00058A3BE016F5F7F4FCE014996F7D28E01AD
:1007F000075F1F4FB801CE014D96F0D28A8591E078
:1008000089278A87AE014F5E5F4FB801CE010196FE
:100810008CDEFED1DC01CB01BC01CD01E4E0A09671
:1008200027C4A0E2B0E0E6E1F4E0F8C3DC01CB01CC
:10083000898F9A8FAB8FBC8F2D8F3E8F4F8F58A390
:10084000BE016F5F7F4FCE014996C8D269E070E06C
:100850006C0F7D1FCE014D96C1D2FE0131966624EC
:1008600077244301130124018981823098F099850E
:10087000923058F420E091818A85981321E02A87EC
:1008800069E070E06C0F7D1FD9C0843059F492305C
:1008900009F45BC020E091818A85981321E02183CF
:1008A000BF01CCC0943009F44DC0823099F392302E
:1008B00009F3ED80FE800F8118852D853E854F85DB
:1008C0005889640153016FE170E00CC0220F331F9F
:1008D000441F551F16950795F794E7946150704093
:1008E00077FD36C0D801C70181709070A070B070DC
:1008F000892BC9F080E090E0220E331E441E551E65
:10090000221633064406550610F481E090E0AA272B
:1009100097FDA095BA2F8A0D9B1DAC1DBD1D680EBD
:10092000791E8A1E9B1EAA0CBB1CCC1CDD1C57FF0B
:10093000CDCF81E090E0A0E0B0E0A82AB92ACA2A91
:10094000DB2AC4CF823009F095CF68E870E076C02A
:10095000228133818B859C85280F391F2E5F3F4F65
:10096000A90160E091818A85981361E06A8B97FE06
:100970000FC02FC0CA010197AC019C01660C771C07
:10098000881C991C57FC41C0220C331C441C551C6C
:1009900090E0691690E0790690E0890690E4990667
:1009A00048F33C8B2B8BD401C3018F779070A070E0
:1009B000B07080349105A105B10581F16D8A7E8A00
:1009C0008F8A988E83E0898B61E170E06C0F7D1FC8
:1009D00035C02F5F3F4FA901D401C30181709070D2
:1009E000A070B070892B61F0569447943794279487
:1009F00080E090E0A0E0B0E8282A392A4A2A5B2A61
:100A00009694879477946794C3CF81E090E0A0E0B8
:100A1000B0E0682A792A8A2A9B2AB6CF67FC05C0EB
:100A2000211431044104510449F280E490E0A0E033
:100A3000B0E0680E791E8A1E9B1EC0CFCB01E8D0A5
:100A4000DC01CB01BC01CD01E2E1A09603C3A8E12A
:100A5000B0E0ECE2F5E0F0C2DC01CB01898B9A8BCF
:100A6000AB8BBC8B2D8B3E8B4F8B588FBE016F5F3A
:100A70007F4FCE014196B2D18E01075F1F4FB80163
:100A8000CE014596ABD18981823018F089858230BC
:100A900018F42FEF3FEF08C0B801CE01019618D22D
:100AA000282F332727FD3095C901E4E06896E0C27E
:100AB000A8E0B0E0EDE5F5E0BDC29B01AC017B0133
:100AC0008C01EE2417FDE394FF2400271127EA820E
:100AD000211531054105510531F482E08983CE01AC
:100AE000019696D043C083E089836EE170E0CB012C
:100AF000EE2031F579018A01A80197012030E0E06C
:100B00003E07E0E04E07E0E45E0798F479018A01D1
:100B1000EE0CFF1C001F111F0197BC01A8019701DB
:100B2000E0E0EE16E0E0FE06E0E00E07E0E41E077F
:100B300068F3ED82FE820F8318877C836B83CFCFAF
:100B40002030E0E03E07E0E04E07E0E85E0741F0DD
:100B5000EE24FF248701E21AF30A040B150BCCCF15
:100B60007C836B8360E070E080E09FECE6E0289699
:100B70007DC2ACE0B0E0EEEBF5E060C2DC01CB01A1
:100B800089879A87AB87BC87BE016F5F7F4FCE0195
:100B9000099624D18981823011F0823028F460E0F6
:100BA00070E080E090E031C0843039F02B813C81EE
:100BB00037FDF5CF2F3131056CF08A81882329F07C
:100BC00060E070E080E090E820C06FEF7FEF8FEF93
:100BD0009FE71BC08EE190E0821B930B2D813E812D
:100BE0004F81588504C056954795379527958A9526
:100BF000D2F78A81882339F0509540953095219518
:100C00003F4F4F4F5F4FCA01B901E2E02C9632C20D
:100C1000A0E0B0E0EDE0F6E007C28824992454019A
:100C2000DC01FC0124813581468157818181082FB7
:100C3000112760E070E08C91823020F46FEF70E05B
:100C40004061A4C0843009F464C0823009F463C0F8
:100C5000211531054105510509F498C0FD01828136
:100C60009381FFEF82389F070CF050C0A2E8EA2E74
:100C7000AFEFFA2EE81AF90A8AE1E816F1040CF04F
:100C80006BC06B0181E090E0A0E0B0E00E2C04C0EE
:100C9000880F991FAA1FBB1F0A94D2F70197A109B9
:100CA000B10982239323A423B5230097A105B1059D
:100CB00019F0F1E0CF2ED12C04C056954795379509
:100CC0002795EA94D2F7C601AA2797FDA095BA2FD7
:100CD000282B392B4A2B5B2BDA01C9018F779070B7
:100CE000A070B07080349105A105B105D1F1215CEF
:100CF0003F4F4F4F5F4F2030E0E03E07E0E04E07B0
:100D0000E0E45E0708F161E070E01EC08038910504
:100D10003CF06FEF70E020E030E040E050E036C0A3
:100D2000BC0161587F4FDA01C9018F779070A070C4
:100D3000B07080349105A105B105D1F0215C3F4F21
:100D40004F4F5F4F57FD1BC097E05695479537951E
:100D500027959A95D1F71AC020E030E040E050E0A6
:100D6000BBCF27FFC8CF205C3F4F4F4F5F4FC3CF54
:100D700027FFE8CF205C3F4F4F4F5F4FE3CF5695A3
:100D80004795379527956F5F7F4FDECF822E932E45
:100D9000942F9F778A2D8078A82EA92A962F979531
:100DA000992797958A2D8F77A82EA92A76956795EA
:100DB000962F9F778B2D8078B82EB92A902F9795F4
:100DC000992797958B2D8F77B82EB92AD501C40115
:100DD000BC01CD01ECE0CDB7DEB742C1CF93DF93CC
:100DE000FC01DB01408151812281622F6F7770E02D
:100DF000221F2227221F9381892F880F822B282FC1
:100E00003327991F9927991FED01998321153105E2
:100E100041F44115510561057105E1F482E08C93BF
:100E200054C02F3F310509F441C02F573040FD0118
:100E30003383228383E08C9387E0440F551F661F22
:100E4000771F8A95D1F77064ED014C835D836E83C3
:100E50007F833BC022E83FEFF901C7E0440F551FF5
:100E6000661F771FCA95D1F783E08C93403080E0EE
:100E7000580780E0680780E4780778F4440F551F2E
:100E8000661F771F21503040F9014030C0E05C07F9
:100E9000C0E06C07C0E47C0788F3ED01FB83EA83C4
:100EA000FD0144835583668377830FC04115510547
:100EB0006105710519F484E08C9307C064FF03C0D9
:100EC00081E08C93C1CF1C92BFCFDF91CF91089569
:100ED0000F931F93CF93DF93FC01DB01808182305E
:100EE00018F09C91923018F461E070E05EC084309C
:100EF000C1F0843001F1943009F447C0823009F424
:100F00004BC0823009F44EC09230A9F04181ED010E
:100F100089814817B9F0442389F08FEF9FEFBC0116
:100F200044C0943031F7EB018981682F77278181A4
:100F3000681B71093AC08181882379F781E090E0CC
:100F4000BC0133C022813381ED018A819B818217EC
:100F500093070CF3281739079CF00481158126812B
:100F60003781FD01648175818681978160177107E2
:100F70008207930780F2061717072807390778F4C6
:100F8000442359F281E090E0DBCFFD018181882389
:100F900021F281E090E0D4CF923009F0B2CF60E04E
:100FA00070E003C0ED018981F2CFCB01DF91CF91D9
:100FB0001F910F910895991B79E004C0991F96170E
:100FC00008F0961B881F7A95C9F78095089597FBBE
:100FD000092E07260AD077FD04D00CD006D00020B9
:100FE0001AF4709561957F4F0895F6F79095819565
:100FF0009F4F0895AA1BBB1B51E107C0AA1FBB1F2F
:10100000A617B70710F0A61BB70B881F991F5A9594
:10101000A9F780959095BC01CD0108952F923F923C
:101020004F925F926F927F928F929F92AF92BF92F8
:10103000CF92DF92EF92FF920F931F93CF93DF93A4
:10104000CDB7DEB7CA1BDB0B0FB6F894DEBF0FBE01
:10105000CDBF09942A88398848885F846E847D844E
:101060008C849B84AA84B984C884DF80EE80FD8050
:101070000C811B81AA81B981CE0FD11D0FB6F894C6
:0A108000DEBF0FBECDBFED010895E5
:10108A003F065B4F666D7D077F6F777C395E7971AE
:10109A0040000000BF86DBCFE6EDFD87FFEFF7FCDF
:1010AA00B9DEF9F1C0808080000000000000000075
:00000001FF
